:1000000000800010CD000000B1060000B306000023
:10001000B5060000B7060000B906000000000000A9
:10002000000000000000000000000000BB0600000F
:10003000BD06000000000000BF060000C106000071
:10004000C3060000C9010000C3060000C30600008B
:10005000C3060000C3060000C3060000C30600007C
:10006000C3060000C3060000C3060000C30600006C
:10007000C3060000C3060000C3060000C30600005C
:10008000C3060000C3060000C3060000C30600004C
:10009000C3060000C3060000C3060000C30600003C
:1000A000C3060000C3060000C3060000C30600002C
:1000B000C3060000C3060000C3060000C30600001C
:1000C000C3060000C3060000C306000001488047C5
:1000D00001480047B93800004547000040F2B0131E
:1000E000C1F200031A780AB901201870704700BFE6
:1000F00040F20000C1F2000008B503682BB140F2E5
:100100000003C0F2000303B1984708BD82B0034664
:100110008DF807304EF20013CEF200039DF9072050
:100120004FEA52129DF8071001F01F014FF0010035
:1001300000FA01F143F8221002B0704782B0034682
:100140008DF807304EF20013CEF200039DF9072020
:100150004FEA52129DF8071001F01F014FF0010005
:1001600000FA01F102F1200243F8221002B07047B8
:1001700082B0034600918DF807309DF90730002BBF
:1001800011DA4EF60053CEF200039DF8072002F07C
:100190000F02A2F10401009AD2B24FEAC202D2B217
:1001A0000B441A760DE04EF20013CEF200039DF9D7
:1001B0000710009AD2B24FEAC202D2B20B4483F8BF
:1001C000002302B0704700BF08B544F20000C4F23B
:1001D00000004FF0000101F013F90346002B5ED040
:1001E00044F20000C4F200004FF0000101F0C4F935
:1001F00040F2B813C1F200031B78012B31D144F255
:100200000000C4F200004FF0000101F07BFB44F25B
:100210000000C4F2000001F0B3FB44F20000C4F29D
:1002200000004FF0010101F06DFB40F2B113C1F28B
:1002300000031B7803F10103DAB240F2B113C1F2FB
:1002400000031A7040F2B113C1F200031B78052BB2
:1002500024D140F2B813C1F200034FF000021A702B
:100260001DE040F2B113C1F200034FF000021A701A
:1002700040F2B913C1F200034FF001021A7044F2C8
:100280000000C4F200004FF0000101F05FFD0246E3
:1002900040F2C413C1F200031A6000E000BF08BDC1
:1002A00008B540F2D813C1F200031B684CF20000FD
:1002B000C4F2000040F20801C1F20001984708BDF5
:1002C00000B589B000F0BCFDFFF7EAFF4FF0030373
:1002D0008DF812304FF000038DF814304FF000030A
:1002E0008DF813304FF001038DF810304FF01A03E2
:1002F0008DF8113004AB184600F062FF4FF0030395
:100300008DF812304FF000038DF814304FF00003D9
:100310008DF813304FF000038DF810304FF00603C6
:100320008DF8113004AB184600F04AFF40F2BC13C0
:10033000C1F200034FF001021A7040F2BC13C1F287
:1003400000034FF001025A6040F2B413C1F20003FF
:100350004FF000021A7040F2B413C1F200034FF0E4
:1003600001025A7040F2B413C1F200034FF00002D0
:100370009A7040F2B413C1F200034FF00102DA7038
:1003800044F20000C4F200004FF0000140F2BC1241
:10039000C1F2000201F064F944F20000C4F200006E
:1003A00040F2B411C1F2000101F050FC44F200002F
:1003B000C4F2000001F0E4FA4FF000038DF81530AC
:1003C0004FF0000306934FF00003ADF8163087E0BE
:1003D0009DF81530002B0DD140F2D813C1F2000367
:1003E0001B684CF20000C4F2000044F2A471C0F299
:1003F0000001984740F2DC13C1F200031B684CF285
:100400000000C4F2000098470346ADF81630BDF86E
:100410001630A3F13003092B49D8BDF81630A3F1EB
:100420003003ADF816309DF8153003F101038DF857
:1004300015309DF81530012B10D1BDF816301A4635
:100440004FEA820213441A464FEA82011A460B46CB
:1004500013444FEA8303ADF816300DE09DF81530D4
:10046000022B09D1BDF816301A464FEA8202134416
:100470004FEA4303ADF81630BDF81630069A134420
:1004800006939DF81530032B0CD140F2D413C1F222
:1004900000031B68069A92B24CF20000C4F20000FE
:1004A000114698474FF00003ADF8163018E040F2BF
:1004B000D813C1F200031B684CF20000C4F2000024
:1004C00044F2D471C0F2000198474FF000038DF858
:1004D00015304FF00003ADF816304FF000030693CF
:1004E0009DF81530022B7FF673AF40F2BC13C1F2BA
:1004F00000034FF001021A7040F2BC13C1F2000376
:100500004FF001025A6040F20000C4F209004FF0BF
:10051000000140F2BC12C1F2000201F0A1F84FF05C
:1005200000038DF804304FF000038DF805304FF0D4
:1005300001038DF807304FF000038DF806304FF0BF
:1005400003038DF808304AF22013C0F20703069A1D
:10055000B3FBF2F3039301AB40F20000C4F20900D5
:10056000194601F043FA40F20000C4F209004FF0CE
:10057000010101F0C7F94FF001004FF00901FFF749
:10058000F7FD4FF00100FFF7C1FD40F2B813C1F2D3
:1005900000034FF001021A7040F2B913C1F20003D8
:1005A0004FF000021A7040F2C413C1F200034FF082
:1005B00000021A6044F20000C4F200004FF0010192
:1005C00001F0A0F940F2D813C1F200031B684CF20D
:1005D0000000C4F2000044F60001C0F20001984798
:1005E00040F2B913C1F200031B78002BF8D040F29F
:1005F000C413C1F200031A6844F24023C0F20F038F
:10060000B3FBF2F3079340F2D413C1F200031B686B
:10061000079A92B24CF20000C4F2000011469847CB
:1006200040F2D813C1F200031B684CF20000C4F280
:10063000000044F61401C0F2000198474FF0010099
:10064000FFF77CFD44F20000C4F2000001F0F6F870
:1006500040F20000C4F2090001F0F0F840F2D813B3
:10066000C1F200031B684CF20000C4F2000044F623
:100670001801C0F20001984740F2DC13C1F20003F8
:100680001B684CF20000C4F2000098470346632B3D
:10069000F2D14BE608B5FFF713FE0346184608BD36
:1006A00082B001900091FEE782B001900091FEE7D8
:1006B000FEE7FEE7FEE7FEE7FEE7FEE7FEE7FEE712
:1006C000FEE7FEE700B583B001900B468DF80330DE
:1006D0000DF10303019819464FF001024FF0010399
:1006E00001F09AFF03B000BD00B585B001904FF056
:1006F00000038DF80F300DF10F03019819464FF0EC
:1007000001024FF0010302F00BF89DF80F3018467C
:1007100005B000BD00B585B001900091009B03932A
:1007200009E0039B1B78039A02F1010203920198EE
:100730001946FFF7C7FF039B1B78002BF1D105B0CB
:1007400000BD00BF00B583B00190009101980099F1
:10075000FFF7E0FF019844F64C01C0F20001FFF7FB
:10076000D9FF03B000BD00BF00B585B001900B46B6
:100770008DF803309DF803204CF6CD43CCF6CC43E6
:10078000A3FB02134FEAD3010B464FEA83030B444A
:100790004FEA4303C3EB02038DF80D309DF80320AD
:1007A0004CF6CD43CCF6CC43A3FB02134FEAD30364
:1007B000DAB24CF6CD43CCF6CC43A3FB02134FEA9E
:1007C000D3010B464FEA83030B444FEA4303C3EBC9
:1007D00002038DF80E309DF8032048F21F53C5F236
:1007E000EB13A3FB02134FEA5313DAB24CF6CD43DB
:1007F000CCF6CC43A3FB02134FEAD3010B464FEADE
:1008000083030B444FEA4303C3EB02038DF80F301D
:100810009DF80F3003F13003DBB201981946FFF762
:1008200051FF9DF80E3003F13003DBB201981946F9
:10083000FFF748FF9DF80D3003F13003DBB201985C
:100840001946FFF73FFF05B000BD00BF00B585B0FA
:1008500001900B46ADF80230BDF802204CF6CD43B6
:10086000CCF6CC43A3FB02134FEAD3010B464FEA6D
:1008700083030B444FEA4303C3EB02039BB28DF89F
:100880000B30BDF802204CF6CD43CCF6CC43A3FB95
:1008900002134FEAD3039AB24CF6CD43CCF6CC43C5
:1008A000A3FB02134FEAD3010B464FEA83030B4429
:1008B0004FEA4303C3EB02039BB28DF80C30BDF843
:1008C000022048F21F53C5F2EB13A3FB02134FEAB9
:1008D00053139AB24CF6CD43CCF6CC43A3FB021390
:1008E0004FEAD3010B464FEA83030B444FEA43031D
:1008F000C3EB02039BB28DF80D30BDF8022044F625
:10090000D353C1F26203A3FB02134FEA93139AB2CB
:100910004CF6CD43CCF6CC43A3FB02134FEAD301F4
:100920000B464FEA83030B444FEA4303C3EB020336
:100930009BB28DF80E30BDF8022041F25973CDF212
:10094000B713A3FB02134FEA53339AB24CF6CD43CD
:10095000CCF6CC43A3FB02134FEAD3010B464FEA7C
:1009600083030B444FEA4303C3EB02039BB28DF8AE
:100970000F309DF80F3003F13003DBB201981946B8
:10098000FFF7A0FE9DF80E3003F13003DBB20198B3
:100990001946FFF797FE9DF80D3003F13003DBB2E7
:1009A00001981946FFF78EFE9DF80C3003F13003D5
:1009B000DBB201981946FFF785FE9DF80B3003F175
:1009C0003003DBB201981946FFF77CFE05B000BD8D
:1009D00000B587B00190009100994CF6CD43CCF65C
:1009E000CC43A3FB01234FEAD30213464FEA830310
:1009F00013444FEA4303C3EB010213468DF80E3054
:100A0000009A4CF6CD43CCF6CC43A3FB02134FEA3D
:100A1000D3014CF6CD43CCF6CC43A3FB01234FEAE4
:100A2000D30213464FEA830313444FEA4303C3EB55
:100A3000010213468DF80F30009A48F21F53C5F299
:100A4000EB13A3FB02134FEA53114CF6CD43CCF644
:100A5000CC43A3FB01234FEAD30213464FEA83039F
:100A600013444FEA4303C3EB010213468DF81030E1
:100A7000009A44F6D353C1F26203A3FB02134FEA78
:100A800093114CF6CD43CCF6CC43A3FB01234FEAA4
:100A9000D30213464FEA830313444FEA4303C3EBE5
:100AA000010213468DF81130009A41F25973CDF2CC
:100AB000B713A3FB02134FEA53314CF6CD43CCF6E8
:100AC000CC43A3FB01234FEAD30213464FEA83032F
:100AD00013444FEA4303C3EB010213468DF812306F
:100AE000009B4FEA531245F6C523C0F67C23A3FBB7
:100AF00002134FEAD3114CF6CD43CCF6CC43A3FB03
:100B000001234FEAD30213464FEA830313444FEA0B
:100B10004303C3EB010213468DF81330009A4DF6E0
:100B20008363C4F21B33A3FB02134FEA93414CF6D9
:100B3000CD43CCF6CC43A3FB01234FEAD3021346AB
:100B40004FEA830313444FEA4303C3EB0102134606
:100B50008DF81430009A4CF66B23C6F65F33A3FB76
:100B600002134FEA93514CF6CD43CCF6CC43A3FB92
:100B700001234FEAD30213464FEA830313444FEA9B
:100B80004303C3EB010213468DF81530009A43F678
:100B90008933C5F2E653A3FB02134FEA53614CF6C7
:100BA000CD43CCF6CC43A3FB01234FEAD30213463B
:100BB0004FEA830313444FEA4303C3EB0102134696
:100BC0008DF81630009B4FEA532244F68333C0F26F
:100BD0000403A3FB02134FEAD3114CF6CD43CCF62A
:100BE000CC43A3FB01234FEAD30213464FEA83030E
:100BF00013444FEA4303C3EB010213468DF8173049
:100C00009DF8173003F13003DBB201981946FFF766
:100C100059FD9DF8163003F13003DBB201981946F7
:100C2000FFF750FD9DF8153003F13003DBB201985A
:100C30001946FFF747FD9DF8143003F13003DBB28E
:100C400001981946FFF73EFD9DF8133003F130037C
:100C5000DBB201981946FFF735FD9DF8123003F11C
:100C60003003DBB201981946FFF72CFD9DF81130D7
:100C700003F13003DBB201981946FFF723FD9DF81D
:100C8000103003F13003DBB201981946FFF71AFD6B
:100C90009DF80F3003F13003DBB201981946FFF7DE
:100CA00011FD9DF80E3003F13003DBB201981946B7
:100CB000FFF708FD07B000BD00B585B001900B46F9
:100CC0008DF80330019844F65001C0F20001FFF79F
:100CD00021FD4FF001038DF80F309DF803209DF8A2
:100CE0000F304FEA830342FA03F3DBB203F00F0342
:100CF0008DF80E309DF80E30092B05D99DF80E3079
:100D000003F13703DBB204E09DF80E3003F130034A
:100D1000DBB201981946FFF7D5FC9DF80F30002B88
:100D20000CBF00230123DBB29DF80F2002F1FF323C
:100D30008DF80F20002BD0D105B000BD00B585B0D7
:100D400001900B46ADF80230019844F65001C0F214
:100D50000001FFF7DFFC4FF003038DF80F30BDF803
:100D600002209DF80F304FEA830342FA03F3DBB20F
:100D700003F00F038DF80E309DF80E30092B05D9C6
:100D80009DF80E3003F13703DBB204E09DF80E301E
:100D900003F13003DBB201981946FFF793FC9DF88D
:100DA0000F30002B0CBF00230123DBB29DF80F2076
:100DB00002F1FF328DF80F20002BD0D105B000BD1D
:100DC00000B585B001900091019844F65001C0F241
:100DD0000001FFF79FFC4FF007038DF80F309DF8DF
:100DE0000F304FEA8303009A22FA03F3DBB203F0D9
:100DF0000F038DF80E309DF80E30092B05D99DF8A4
:100E00000E3003F13703DBB204E09DF80E3003F13E
:100E10003003DBB201981946FFF754FC9DF80F3000
:100E2000002B0CBF00230123DBB29DF80F2002F141
:100E3000FF328DF80F20002BD1D105B000BD00BFCF
:100E400000B585B04FF001038DF802304FF000037C
:100E50008DF804304FF000038DF803304FF002039B
:100E60008DF801304FF000038DF800306B461846C6
:100E700000F0A6F94FF003038DF801306B461846D9
:100E800000F09EF902AB184601F03EFB4FF4E1334F
:100E9000029302AB4CF20000C4F20000194601F0CC
:100EA00025F94CF20000C4F200004FF0010102F0FD
:100EB00039F840F2D813C1F2000340F21572C0F2C3
:100EC00000021A6040F2E013C1F2000340F24572E2
:100ED000C0F200021A6040F2E413C1F2000340F2D3
:100EE000C562C0F200021A6040F2E813C1F20003CA
:100EF00040F6B942C0F200021A6040F2EC13C1F2AF
:100F0000000340F63D52C0F200021A6040F2D013D6
:100F1000C1F2000340F6C152C0F200021A6040F272
:100F2000C813C1F2000340F26972C0F200021A60F5
:100F300040F2D413C1F2000340F64D02C0F20002A9
:100F40001A6040F2CC13C1F2000340F6D112C0F295
:100F500000021A6040F2DC13C1F2000340F2E962C1
:100F6000C0F200021A6005B000BD00BF86B0134693
:100F700002468DF807200A468DF806208DF80530C8
:100F80009DF8063003939DF807304FEA430304931E
:100F90004CF20003C4F202030593039B0F2B07D905
:100FA000039BA3F110030393049B03F10103049338
:100FB000049B4FEA8302059B1344049A4FEA820183
:100FC000059A0A441168039A4FEA42024FF003005F
:100FD00000FA02F26FEA020201EA02021A60049BBE
:100FE0004FEA8302059B1344049A4FEA8201059A53
:100FF0000A4411689DF80500039A4FEA420200FA7C
:1010000002F241EA02021A6006B0704786B0134647
:1010100002468DF807200A468DF806208DF8053027
:101020009DF8063003939DF807304FEA430304937D
:101030004CF24003C4F202030593039B0F2B07D924
:10104000039BA3F110030393049B03F10103049397
:10105000049B4FEA8302059B1344049A4FEA8201E2
:10106000059A0A441168039A4FEA42024FF00300BE
:1010700000FA02F26FEA020201EA02021A60049B1D
:101080004FEA8302059B1344049A4FEA8201059AB2
:101090000A4411689DF80500039A4FEA420200FADB
:1010A00002F241EA02021A6006B0704784B01346A9
:1010B00002468DF807200A468DF806208DF8053087
:1010C0004CF26803C4F2020303939DF80530012B30
:1010D00016D19DF807304FEA8302039B13449DF815
:1010E00007204FEA8201039A0A4411689DF80620FE
:1010F0004FF0010000FA02F241EA02021A6017E022
:101100009DF807304FEA8302039B13449DF80720A4
:101110004FEA8201039A0A4411689DF806204FF0B5
:10112000010000FA02F26FEA020201EA02021A600A
:1011300004B0704782B003468DF807309DF8073041
:10114000012B0CD14CF20003C4F202034CF200025A
:10115000C4F20202926A42F008029A620FE09DF81D
:101160000730002B0BD14CF20003C4F202034CF207
:101170000002C4F20202926A22F008029A6202B0ED
:10118000704700BF84B002460B468DF807208DF8EB
:1011900006309DF80730012B02D14FF00503039371
:1011A0009DF80630002B02D14FF00A0303934CF256
:1011B0000003C4F20203039ADA6704B0704700BF69
:1011C00000B583B00190019B1978019B5A78019B6F
:1011D0009B78084611461A46FFF7C8FE019B19780E
:1011E000019B5A78019BDB78084611461A46FFF7A7
:1011F0000DFF019B1978019B5A78019B1B790846CA
:1012000011461A46FFF752FF03B000BD00B585B086
:101210000190019B032B26D801A252F823F000BFB6
:10122000311200003F1200004D1200005B1200005E
:101230004FF0020002F0DEFC0346039313E04FF090
:10124000040002F0D7FC034603930CE04FF02C009F
:1012500002F0D0FC0346039305E04FF02E0002F0AD
:10126000C9FC03460393039B184605B000BD00BFAD
:1012700000B585B0019000910198FFF7C7FF0346C4
:101280001A464FF00003CDE90223009B1A464FF0A7
:101290000003029903FB01F1039802FB00F00144F3
:1012A0000298A0FB022319440B46104619464FF43E
:1012B000742202F510724FF0000302F04BFD02465B
:1012C0000B46CDE90223029B184605B000BD00BFC6
:1012D00084B001904FF0FF330393019A44F200036E
:1012E000C4F200039A4203D14FF0000303931FE0BE
:1012F000019A48F20003C4F200039A4203D14FF06E
:101300000103039314E0019A40F20003C4F20903BD
:101310009A4203D14FF00203039309E0019A44F289
:101320000003C4F209039A4202D14FF0030303936E
:10133000039B184604B0704700B585B001900B467A
:101340008DF80330019A44F20003C4F200039A427C
:101350001CD0019A48F20003C4F200039A4215D04F
:10136000019A40F20003C4F209039A420ED0019A96
:1013700044F20003C4F209039A4207D044F6540031
:10138000C0F200004FF0A601FFF78AF99DF8033084
:10139000002B1BD09DF80330012B17D09DF8033094
:1013A000022B13D09DF80330032B0FD09DF8033090
:1013B000042B0BD09DF80330052B07D044F65400C6
:1013C000C0F200004FF0A701FFF76AF9019B1B680C
:1013D000DAB29DF803304FF0010101FA03F3DBB2FA
:1013E00002EA03038DF80F309DF80F30002B02D076
:1013F0004FF0010301E04FF00003184605B000BDB7
:1014000000B585B001900B468DF80330019A44F287
:101410000003C4F200039A421CD0019A48F2000370
:10142000C4F200039A4215D0019A40F20003C4F2BC
:1014300009039A420ED0019A44F20003C4F2090350
:101440009A4207D044F65400C0F200004FF0C401A5
:10145000FFF726F99DF80330002B1BD09DF80330D1
:10146000012B17D09DF80330022B13D09DF80330C9
:10147000032B0FD09DF80330042B0BD09DF80330C5
:10148000052B07D044F65400C0F200004FF0C50110
:10149000FFF706F9019B1B68DAB29DF8033003F1F0
:1014A00004034FF0010101FA03F3DBB202EA030384
:1014B0008DF80F309DF80F30002B02D04FF0010354
:1014C00001E04FF00003184605B000BD00B583B041
:1014D00001900B468DF80330019A44F20003C4F2E8
:1014E00000039A421CD0019A48F20003C4F20003A0
:1014F0009A4215D0019A40F20003C4F209039A42BD
:101500000ED0019A44F20003C4F209039A4207D0B4
:1015100044F65400C0F200004FF0DD01FFF7C0F8C0
:101520009DF80330002B1BD09DF80330012B17D002
:101530009DF80330022B13D09DF80330032B0FD0FE
:101540009DF80330042B0BD09DF80330052B07D0FA
:1015500044F65400C0F200004FF0DE01FFF7A0F89F
:101560009DF803304FF0010202FA03F31A46019B83
:101570001A6003B000BD00BF00B583B001900B46F8
:101580008DF80330019A44F20003C4F200039A423A
:101590001CD0019A48F20003C4F200039A4215D00D
:1015A000019A40F20003C4F209039A420ED0019A54
:1015B00044F20003C4F209039A4207D044F65400EF
:1015C000C0F200004FF0F401FFF76AF89DF8033015
:1015D000002B1BD09DF80330012B17D09DF8033052
:1015E000022B13D09DF80330032B0FD09DF803304E
:1015F000042B0BD09DF80330052B07D044F6540084
:10160000C0F200004FF0F501FFF74AF89DF80330F3
:1016100003F104034FF0010202FA03F31A46019B9F
:101620001A6003B000BD00BF84B0034600918DF87E
:1016300007309DF80730002B0AD1009B0293029BD4
:101640004FF001021A70029B4FF001025A6005E050
:10165000009B0393039B4FF000025A7004B0704745
:1016600000B587B003900B4601928DF80B30039ABA
:1016700044F20003C4F200039A421CD0039A48F2D9
:101680000003C4F200039A4215D0039A40F200030B
:10169000C4F209039A420ED0039A44F20003C4F242
:1016A00009039A4207D044F65400C0F2000040F209
:1016B0002B11FEF7F5FF9DF80B30002B13D09DF892
:1016C0000B30012B0FD09DF80B30012B0BD09DF868
:1016D0000B30012B07D044F65400C0F200004FF449
:1016E0009671FEF7DDFF039A44F20003C4F2000393
:1016F0009A420CD14FF002004FF0010102F0AEFA15
:101700004FF002004FF0000102F0EEF93AE0039AC8
:1017100048F20003C4F200039A420CD14FF00400D7
:101720004FF0010102F09AFA4FF004004FF000016F
:1017300002F0DAF926E0039A40F20003C4F209034A
:101740009A420CD14FF480004FF0010102F086FA6A
:101750004FF02C004FF0000102F0C6F912E0039A9E
:1017600044F20003C4F209039A420BD14FF4000083
:101770004FF0010102F072FA4FF02E004FF000011D
:1017800002F0B2F9039B9B6A23F00302039B9A6267
:10179000039B9A6A039B9A62039B4FF000029A6034
:1017A000039B4FF000021A61039B4FF00002DA60C6
:1017B000039B5B6843F00202039B5A60039B5B68D8
:1017C00023F00202039B5A609DF80B30002B1CD1C2
:1017D000019B0493049B1B78002B06D1049B5B6840
:1017E00003F1FF32039BDA6021E00398FFF770FDFD
:1017F0000246049B5B6810461946FFF739FD034615
:1018000003F1FF32039BDA6011E0019B0593039B18
:101810009B6A23F00C02039B9A62059B5B78012B69
:1018200005D1039B9B6A43F00402039B9A62039BCE
:101830004FF0FF321A6007B000BD00BF00B583B0A3
:101840000190019A44F20003C4F200039A421CD0B2
:10185000019A48F20003C4F200039A4215D0019A9B
:1018600040F20003C4F209039A420ED0019A44F2F6
:101870000003C4F209039A4207D044F65400C0F2B0
:10188000000040F27911FEF70BFF019B4FF00002C0
:101890005A60019A44F20003C4F200039A4206D14E
:1018A0004FF002004FF0000102F0D8F928E0019A51
:1018B00048F20003C4F200039A4206D14FF004003C
:1018C0004FF0000102F0CAF91AE0019A40F2000359
:1018D000C4F209039A4206D14FF480004FF0000190
:1018E00002F0BCF90CE0019A44F20003C4F20903CF
:1018F0009A4205D14FF480004FF0000102F0AEF99A
:1019000003B000BD00B583B001900B468DF80330E5
:10191000019A44F20003C4F200039A421CD0019AD7
:1019200048F20003C4F200039A4215D0019A40F233
:101930000003C4F209039A420ED0019A44F2000354
:10194000C4F209039A4207D044F65400C0F20000E2
:101950004FF4CD71FEF7A4FE9DF80330012B06D1A4
:10196000019B5B6843F00102019B5A6005E0019B0B
:101970005B6823F00102019B5A6003B000BD00BF09
:1019800000B583B00190019A44F20003C4F2000351
:101990009A421CD0019A48F20003C4F200039A4212
:1019A00015D0019A40F20003C4F209039A420ED006
:1019B000019A44F20003C4F209039A4207D044F6A4
:1019C0005400C0F200004FF4D971FEF769FE019B8C
:1019D0005B6843F00202019B5A60019B5B6823F045
:1019E0000202019B5A6003B000BD00BF00B583B086
:1019F00001900091019A44F20003C4F200039A425C
:101A00001CD0019A48F20003C4F200039A4215D098
:101A1000019A40F20003C4F209039A420ED0019ADF
:101A200044F20003C4F209039A4207D044F654007A
:101A3000C0F2000040F2D111FEF732FE009B1B798C
:101A4000002B13D0009B1B79012B0FD0009B1B791F
:101A5000022B0BD0009B1B79032B07D044F65400BC
:101A6000C0F200004FF4E971FEF71AFE009B1B78EC
:101A7000032B1FD801A252F823F000BF8D1A0000DB
:101A8000971A0000A11A0000AB1A0000009B9A6888
:101A9000019B9A610FE0009B9A68019BDA610AE062
:101AA000009B9A68019B1A6205E0009B9A68019B63
:101AB0005A6200E0FEE7019B5969009B1B781A46B9
:101AC00013464FEA430313444FF0070202FA03F3AD
:101AD0006FEA030301EA0302019B5A61009B5B78F2
:101AE000002B10D0019B5969009B1B781A461346A6
:101AF0004FEA430313444FF0010202FA03F341EAB1
:101B00000302019B5A61009BDB78002B12D0019BE2
:101B10005969009B1B781A4613464FEA4303134446
:101B200003F101034FF0010202FA03F341EA030259
:101B3000019B5A61009B9B78002B12D0019B596935
:101B4000009B1B781A4613464FEA4303134403F1E4
:101B500002034FF0010202FA03F341EA0302019B80
:101B60005A61019BDA6B009B1B784FEA430303F138
:101B700004034FF0030101FA03F36FEA030302EADF
:101B80000302019BDA63019BDA6B009B1B7903F074
:101B90000301009B1B784FEA430303F1040301FA9E
:101BA00003F342EA0302019BDA6303B000BD00BF06
:101BB00000B585B003900B4601928DF80B30039A67
:101BC00044F20003C4F200039A421CD0039A48F284
:101BD0000003C4F200039A4215D0039A40F20003B6
:101BE000C4F209039A420ED0039A44F20003C4F2ED
:101BF00009039A4207D044F65400C0F2000040F2B4
:101C00000721FEF74DFD9DF80B30032B1BD801A2D9
:101C100052F823F0251C00002D1C0000351C00008C
:101C20003D1C0000039B019A9A610DE0039B019A01
:101C3000DA6109E0039B019A1A6205E0039B019AAD
:101C40005A6200BF00E0FEE705B000BD00B583B0FA
:101C500001900091019A44F20003C4F200039A42F9
:101C60001CD0019A48F20003C4F200039A4215D036
:101C7000019A40F20003C4F209039A420ED0019A7D
:101C800044F20003C4F209039A4207D044F6540018
:101C9000C0F2000040F22D21FEF702FD019B996A7F
:101CA000009B1B781A4613464FEA430313444FF038
:101CB000070202FA03F36FEA030301EA0302019B3E
:101CC0009A62009B5B78002B10D0019B996A009B65
:101CD0001B781A4613464FEA430313444FF00102A0
:101CE00002FA03F341EA0302019B9A62009B9B788C
:101CF000002B12D0019B996A009B1B781A46134651
:101D00004FEA4303134403F101034FF0010202FAC7
:101D100003F341EA0302019B9A62009BDB78002BEC
:101D200012D0019B996A009B1B781A4613464FEA12
:101D30004303134403F102034FF0010202FA03F3D9
:101D400041EA0302019B9A6203B000BD00B583B073
:101D500001900B468DF80330019A44F20003C4F25F
:101D600000039A421CD0019A48F20003C4F2000317
:101D70009A4215D0019A40F20003C4F209039A4234
:101D80000ED0019A44F20003C4F209039A4207D02C
:101D900044F65400C0F200004FF41271FEF780FCCC
:101DA0009DF80330002B0BD09DF80330012B07D09A
:101DB00044F65400C0F2000040F24921FEF770FCE6
:101DC0009DF80330002B02D1019BDB6A01E0019BEF
:101DD0001B6B184603B000BD2DE9F04F95B0039082
:101DE00002914FF000038DF81730039A4CF2000374
:101DF000C4F200039A4206D14FF0060001F0FAFE49
:101E00000346069328E0039A40F20003C4F201035C
:101E10009A4206D14FF0080001F0ECFE034606930B
:101E20001AE0039A48F20003C4F209039A4206D169
:101E30004FF0300001F0DEFE034606930CE0039AFB
:101E40004CF20003C4F209039A4205D14FF032006C
:101E500001F0D0FE034606934FF0FF3312934FF08C
:101E6000000309934FF000030A934FF000024FF074
:101E70000003CDE90C234FF00103089374E04FF009
:101E80000003079363E0069B1A464FF000034FEAF6
:101E900012114FEA037541EA05054FEA0274089BE7
:101EA0001A464FF0000302FB05F104FB03F0014466
:101EB000A4FB022319440B46089807990144029891
:101EC00000FB01F18A464FF0000BCDE900AB104654
:101ED0001946DDE9002301F03DFF02460B46CDE93E
:101EE0000E230E9B11930F9B9A464FF0000B534607
:101EF0000B93119BB3F1004F07D9119BC3F1000362
:101F000011930B9B03F101030B930B9B002B17D039
:101F10000B9BB3F5803F15D8119A129B9A4212D2AF
:101F2000119B12930B9B1A464FF00003CDE90C2333
:101F3000079B0993089B0A93129B002B0CD002E08D
:101F400000BF00E000BF079B03F101030793079A5E
:101F5000089B9A4297D300E000BF129B002B07D04A
:101F6000089B03F101030893089B0F2B87D900E01E
:101F700000BFDDE90C2352EA030B02D14FF000034E
:101F8000AFE0069B4FEA13130A9A02FB03F31C46C9
:101F90004FF000050A9A099B13441A464FF00003BC
:101FA0000C9903FB01F10D9802FB00F001440C9821
:101FB000A0FB022319440B462046294601F0CAFE25
:101FC00002460B4613461393029A139B9A4205D975
:101FD000029A139BC3EB0203129304E0139A029B31
:101FE000C3EB02031293129B4FF0640202FB03F255
:101FF000029BB2FBF3F31293129B022B6FD8039A4E
:1020000040F20003C4F201039A4232D1039A039BC7
:102010001B7BDBB26FEA43636FEA5363DBB213737C
:10202000039B0D9A4FEA02620C994FEA112842EA8B
:1020300008080D9A4FEA12295FFA88F21A71039B79
:102040009DF830201A70039A039B1B7BDBB203F0D0
:102050007F031373039B0A9A4FEA021202F0FF01F7
:10206000099A02F00F0241EA020202F0FF029A62AC
:1020700031E0039B1B7BDBB26FEA43636FEA536380
:10208000DAB2039B1A730D9B4FEA03630C9A4FEA73
:10209000122643EA06060D9B4FEA1327F2B2039B72
:1020A0001A719DF83020039B1A70039B1B7BDBB2D7
:1020B00003F07F03039A13730A9BDBB24FEA031307
:1020C000DAB2099BDBB203F00F0342EA0303DAB290
:1020D000039B83F828204FF001038DF817309DF8FB
:1020E0001730184615B0BDE8F08F00BF00B585B0B9
:1020F00001900091019A4CF20003C4F200039A424D
:102100001CD0019A40F20003C4F201039A4215D098
:10211000019A48F20003C4F209039A420ED0019AD0
:102120004CF20003C4F209039A4207D044F664005B
:10213000C0F200004FF0CA01FEF7B2FA009B5B79D3
:10214000002B13D0009B5B79012B0FD0009B5B7998
:10215000022B0BD0009B5B79032B07D044F6640065
:10216000C0F200004FF0CB01FEF79AFA009B9B797A
:10217000002B0BD0009B9B79012B07D044F6640009
:10218000C0F200004FF0CC01FEF78AFA009B1B79E9
:10219000002B17D0009B1B79012B13D0009B1B79C0
:1021A000022B0FD0009B1B79032B0BD0009B1B79BC
:1021B000042B07D044F66400C0F200004FF0CD01BC
:1021C000FEF76EFA019A4CF20003C4F200039A4241
:1021D00005D14FF008004FF0010101F03FFD019AD9
:1021E00040F20003C4F201039A4205D14FF01000FF
:1021F0004FF0010101F032FD019A48F20003C4F2F0
:1022000009039A4205D14FF080704FF0010101F0AF
:1022100025FD019A4CF20003C4F209039A4205D14C
:102220004FF000704FF0010101F018FD019A40F2EB
:102230000003C4F201039A424DD1019B4FF0070203
:102240001A72019B4FF000021A7203E0019B1B7887
:10225000DBB20393019B1B7DDBB203F00103DBB216
:10226000002BF3D1019B6FF07F0283F83020019B9C
:102270001B7DDBB203F02003002BF8D0019B4FF055
:10228000000283F83020019B4FF000025A60019B4E
:102290004FF000021A73019B4FF000021A62019B7B
:1022A0004FF000021A74019B4FF0000283F84C209B
:1022B000019B4FF0000283F85420019B4FF0000275
:1022C00083F85020019B1B7EDBB20393019B1B7D97
:1022D000DBB2039335E0019B4FF007021A72019BBA
:1022E0004FF000021A7203E0019B1B78DBB20393EC
:1022F000019B1B7DDBB203F00103DBB2002BF3D1AA
:10230000019B6FF07F0283F83020019B1B7DDBB2C5
:1023100003F02003002BF8D0019B4FF0000283F85C
:102320003020019B4FF000025A60019B4FF00002E9
:102330001A73019B4FF000021A62019B1B7DDBB2F6
:102340000393019A4CF20003C4F209039A4204D1A8
:10235000019B4FF0000283F82420009B1B6801982A
:102360001946FFF739FD019A40F20003C4F2010358
:102370009A4206D1019B1B7BDBB203F0C00303939F
:1023800005E0019B1B7BDBB203F0C0030393009BC2
:102390005B79012B04D0022B07D0002B0FD009E072
:1023A000039B43F0010303930AE0039B43F0020302
:1023B000039305E0039B43F00303039300E000BF96
:1023C000009B1B79002B23D0039B43F0080303934E
:1023D000009B1B7903F1FF33032B19D801A252F89C
:1023E00023F000BF11240000F5230000FF230000AC
:1023F00009240000039B43F01003039308E0039BB0
:1024000043F02003039303E0039B43F03003039363
:10241000009B9B79012B03D1039B43F0040303939F
:10242000019A40F20003C4F201039A4204D1019BD5
:10243000039AD2B21A7303E0039BDAB2019B1A73B8
:1024400005B000BD00B583B00190019A4CF20003C5
:10245000C4F200039A421CD0019A40F20003C4F275
:1024600001039A4215D0019A48F20003C4F209030D
:102470009A420ED0019A4CF20003C4F209039A4228
:1024800007D044F66400C0F200004FF4CB71FEF7B1
:1024900007F901984FF0000100F044FD019A4CF259
:1024A0000003C4F200039A4205D14FF008004FF038
:1024B000000101F0D3FB019A40F20003C4F20103D2
:1024C0009A4205D14FF010004FF0000101F0C6FB19
:1024D000019A48F20003C4F209039A4205D14FF071
:1024E00080704FF0000101F0B9FB019A4CF200033B
:1024F000C4F209039A4205D14FF000704FF0000179
:1025000001F0ACFB03B000BD82B00190019B4FF421
:1025100016521A60019B4FF003025A71019B4FF053
:1025200000021A71019B4FF000029A7102B07047CD
:1025300000B583B001900B468DF80330019A4CF240
:102540000003C4F200039A421CD0019A40F2000337
:10255000C4F201039A4215D0019A48F20003C4F272
:1025600009039A420ED0019A4CF20003C4F2090307
:102570009A4207D044F66400C0F200004FF4ED71B7
:10258000FEF78EF8019A40F20003C4F201039A426A
:1025900004D1019B9DF803201A7003E0019B9DF874
:1025A00003201A7003B000BD00B583B00190019AFA
:1025B0004CF20003C4F200039A421CD0019A40F28C
:1025C0000003C4F201039A4215D0019A48F20003B5
:1025D000C4F209039A420ED0019A4CF20003C4F2ED
:1025E00009039A4207D044F66400C0F2000040F2AA
:1025F000F311FEF755F8019A40F20003C4F201030B
:102600009A4203D1019B1B78DBB202E0019B1B784D
:10261000DBB2184603B000BD00B58BB00390029149
:1026200001928DF80330029B0993019B05939DF85D
:102630000330012B3ED14FF00003069336E04FF0FC
:10264000FF33079306E0079B002B0BD0079B03F19A
:10265000FF330793039B1B7DDBB203F02003002BAA
:10266000F1D000E000BF079B002B52D04FF01003C9
:10267000089315E0099B1B78099A02F1010209925F
:1026800003981946FFF754FF089B03F1FF330893A3
:10269000059B03F1FF330593069B03F101030693AA
:1026A000089B002B02D0059B002BE3D1059B002B40
:1026B000C5D131E04FF00003069326E0039B1B7D5C
:1026C000DBB203F02003002B25D04FF0100308935A
:1026D00015E0099B1B78099A02F1010209920398FF
:1026E0001946FFF725FF059B03F1FF330593089B70
:1026F00003F1FF330893069B03F101030693089B44
:10270000002B02D0059B002BE3D1059B002BD5D1DC
:1027100002E000BF00E000BF069B18460BB000BD02
:1027200000B589B00390029101928DF80330029BAD
:102730000793019B04939DF80330012B31D14FF097
:102740000003059329E04FF0FF33069306E0069B54
:10275000002B0BD0069B03F1FF330693039B1B7DDD
:10276000DBB203F00103002BF1D000E000BF069BB9
:10277000002B38D00398FFF717FF03461A46079B34
:102780001A70079B03F101030793049B03F1FF33C6
:102790000493059B03F101030593049B002BD2D105
:1027A00024E04FF00003059319E0039B1B7DDBB28F
:1027B00003F00103002B18D00398FFF7F5FE034642
:1027C0001A46079B1A70079B03F101030793059BA9
:1027D00003F101030593049B03F1FF330493049B6E
:1027E000002BE2D102E000BF00E000BF059B1846CD
:1027F00009B000BD00B583B00190019A4CF200030E
:10280000C4F200039A421CD0019A40F20003C4F2C1
:1028100001039A4215D0019A48F20003C4F2090359
:102820009A420ED0019A4CF20003C4F209039A4274
:1028300007D044F66400C0F2000040F28521FDF7A5
:102840002FFF019A40F20003C4F201039A4208D11B
:10285000019B019A127BD2B242F04002D2B21A73AB
:1028600007E0019B1B7BDBB243F04003DAB2019B24
:102870001A7303B000BD00BF00B585B001901346C8
:102880000A468DF803208DF80230019A4CF20003BD
:10289000C4F200039A421CD0019A40F20003C4F231
:1028A00001039A4215D0019A48F20003C4F20903C9
:1028B0009A420ED0019A4CF20003C4F209039A42E4
:1028C00007D044F66400C0F200004FF42B71FDF70E
:1028D000E7FE9DF80230002B0BD09DF80230012B53
:1028E00007D044F66400C0F2000040F2AD21FDF7CD
:1028F000D7FE9DF80330062B2BD801A252F823F007
:102900001D290000252900002D290000352900007F
:102910003D290000452900004D2900004FF001032A
:10292000039316E04FF00203039312E04FF0040309
:1029300003930EE04FF0080303930AE04FF0800387
:10294000039306E04FF48073039302E04FF40073A7
:102950000393019A40F20003C4F201039A4224D186
:102960009DF80330002B3CD09DF80330012B38D06C
:102970009DF80330022B34D09DF80330052B30D066
:102980009DF80330062B2CD09DF80330032B28D064
:102990009DF80330042B24D044F66400C0F20000FC
:1029A00040F2C921FDF77CFE1BE09DF80330002BAF
:1029B00017D09DF80330012B13D09DF80330022B64
:1029C0000FD09DF80330052B0BD09DF80330062B5C
:1029D00007D044F66400C0F2000040F2CD21FDF7BC
:1029E0005FFE9DF80230012B16D1019A40F20003E0
:1029F000C4F201039A4207D1019B019A5168039ADC
:102A000041EA02025A602DE0019B5A68039B42EAA8
:102A10000302019B5A6025E0019A40F20003C4F2D0
:102A200001039A420FD1019A019B5968039B6FEAF7
:102A3000030301EA030140F28F33C0F2000301EA0D
:102A4000030353600EE0019B5A68039B6FEA030384
:102A500002EA030240F20733C0F2000302EA030372
:102A6000019A536005B000BD00B583B00190019A92
:102A70004CF20003C4F200039A421CD0019A40F2C7
:102A80000003C4F201039A4215D0019A48F20003F0
:102A9000C4F209039A420ED0019A4CF20003C4F228
:102AA00009039A4207D044F66400C0F2000040F2E5
:102AB000FB21FDF7F5FD019A40F20003C4F201038A
:102AC0009A4206D140F20003C4F201031B7DDBB23F
:102AD00002E0019B1B7DDBB2184603B000BD00BFC6
:102AE00000B583B00190019A4CF20003C4F20003D8
:102AF0009A421CD0019A40F20003C4F201039A42A8
:102B000015D0019A48F20003C4F209039A420ED08C
:102B1000019A4CF20003C4F209039A4207D044F62A
:102B20006400C0F2000040F21231FDF7B9FD019BD4
:102B30009A6840F2CF33C0F2000302EA030318465A
:102B400003B000BD82B00190019B1B7DDBB203F09E
:102B50004003002B02D04FF0000301E04FF00103CF
:102B6000184602B0704700BF00B585B001900091D3
:102B70004FF000038DF80F30019A4CF20003C4F2BD
:102B800000039A421CD0019A40F20003C4F20103F0
:102B90009A4215D0019A48F20003C4F209039A42FE
:102BA0000ED0019A4CF20003C4F209039A4207D0F6
:102BB00044F66400C0F200004FF44E71FDF770FD62
:102BC000009BDB78002B13D0009BDB78012B0FD010
:102BD000009BDB78022B0BD0009BDB78032B07D00C
:102BE00044F66400C0F2000040F23931FDF758FDB0
:102BF000009B9B78002B0BD0009B9B78012B07D070
:102C000044F66400C0F2000040F23A31FDF748FD9E
:102C1000009B1B78002B0BD0009B1B78012B07D04F
:102C200044F66400C0F2000040F23B31FDF738FD8D
:102C3000009B5B78002B0BD0009B5B78012B07D0AF
:102C400044F66400C0F200004FF44F71FDF728FD18
:102C50009DF80F3043F001038DF80F30009BDB78B7
:102C6000012B04D0022B09D0002B19D00FE09DF8C6
:102C70000F3043F040038DF80F3012E09DF80F3015
:102C80006FEA43636FEA53638DF80F3009E09DF8F4
:102C90000F306FEA83636FEA93638DF80F3000E0C3
:102CA00000BF009B5B78012B05D19DF80F3043F0EE
:102CB00004038DF80F30009B1B78012B05D19DF884
:102CC0000F3043F002038DF80F30009B9B78012BEF
:102CD00005D19DF80F3043F008038DF80F30019AAD
:102CE00040F20003C4F201039A4206D1019A9DF812
:102CF0000F3003F0CF03137205E09DF80F3003F09F
:102D0000CF03019A137205B000BD00BF82B00190DD
:102D1000019B4FF000029A70019B4FF00002DA70A5
:102D2000019B4FF001021A70019B4FF001025A7093
:102D300002B0704700B587B00390029113468DF83A
:102D40000730039A4CF20003C4F200039A421CD0ED
:102D5000039A40F20003C4F201039A4215D0039A89
:102D600048F20003C4F209039A420ED0039A4CF2CF
:102D70000003C4F209039A4207D044F66400C0F28B
:102D8000000040F29331FDF78BFC9DF80730002BDB
:102D90000BD09DF80730012B07D044F66400C0F239
:102DA00000004FF46571FDF77BFC4FF000030593C5
:102DB0009DF80730012B0FD1029B1B78012B03D10B
:102DC000059B43F002030593029B5B78012B03D123
:102DD000059B43F004030593039A40F20003C4F2F9
:102DE00001039A422BD19DF80730012B22D1039A7F
:102DF000039B1B7BDBB26FEA43636FEA5363DBB277
:102E00001373039B4FF000021A70039B4FF00002F4
:102E10001A71039A039B1B7BDBB203F07F031373CE
:102E2000039B4FF010029A62039B059A42F0010245
:102E30001A6230E0039B4FF000021A622BE09DF80B
:102E40000730012B23D1039B1B7BDBB26FEA43636B
:102E50006FEA5363DAB2039B1A73039B4FF00002CD
:102E60001A70039B4FF000021A71039B1B7BDBB2AD
:102E700003F07F03039A1373039B4FF0100283F850
:102E80002820059B43F00102039B1A6203E0039B89
:102E90004FF000021A6207B000BD00BF00B583B05A
:102EA00001900B46ADF80230019A4CF20003C4F2D7
:102EB00000039A421CD0019A40F20003C4F20103BD
:102EC0009A4215D0019A48F20003C4F209039A42CB
:102ED0000ED0019A4CF20003C4F209039A4207D0C3
:102EE00044F66400C0F200004FF47571FDF7D8FBA2
:102EF000019A40F20003C4F201039A4208D1019BF7
:102F00001A6ABDF8023042EA0302019B1A6207E026
:102F1000019B1A6ABDF8023042EA0302019B1A6261
:102F200003B000BD00B583B001900B468DF80330AF
:102F3000019A4CF20003C4F200039A421CD0019A99
:102F400040F20003C4F201039A4215D0019A48F2FC
:102F50000003C4F209039A420ED0019A4CF2000316
:102F6000C4F209039A4207D044F66400C0F200009C
:102F700040F2EB31FDF794FB9DF80330002B0BD0B2
:102F80009DF80330012B07D044F66400C0F2000026
:102F90004FF47B71FDF784FB9DF80330012B20D1AA
:102FA000019A40F20003C4F201039A420CD1019A43
:102FB000019B93F83030DBB26FEA43636FEA5363EF
:102FC000DBB282F8303024E0019B93F83030DBB282
:102FD0006FEA43636FEA5363DAB2019B83F83020F0
:102FE00017E0019A40F20003C4F201039A4208D1AB
:102FF000019B93F83030019B4FF0000283F83020A2
:1030000007E0019B93F83030019B4FF0000283F8FA
:10301000302003B000BD00BF00B583B001900B4667
:103020008DF80330019A4CF20003C4F209039A426E
:1030300007D044F66400C0F2000040F21541FDF7ED
:103040002FFB9DF80330002B0BD09DF80330012B94
:1030500007D044F66400C0F2000040F21641FDF7CC
:103060001FFB9DF80330012B0AD1019B93F82430FC
:10307000DBB243F00203DAB2019B83F824200CE0B8
:103080009DF80330002B08D1019B93F82430DBB26C
:1030900003F03D03019A82F8243003B000BD00BF65
:1030A00000B583B001900B468DF80330019A4CF2C5
:1030B0000003C4F209039A4207D044F66400C0F248
:1030C000000040F22D41FDF7EBFA9DF80330002B94
:1030D0000BD09DF80330012B07D044F66400C0F2FA
:1030E000000040F22E41FDF7DBFA9DF80330012B82
:1030F0000AD1019B93F82430DBB243F00103DAB22A
:10310000019B83F8242008E0019B93F82430DBB274
:1031100003F03E03019A82F8243003B000BD00BFE3
:1031200000B585B001900B468DF80330019A4CF242
:103130000003C4F209039A4207D044F66400C0F2C7
:10314000000040F24E41FDF7ABFA9DF80330002B32
:1031500023D09DF80330012B1FD09DF80330022BA4
:103160001BD09DF80330032B17D09DF80330042BA0
:1031700013D09DF80330052B0FD09DF80330062B9C
:103180000BD09DF80330072B07D044F66400C0F243
:10319000000040F24F41FDF783FA9DF8033003F041
:1031A00007034FEAC3030393019B93F82430DBB278
:1031B00023F038030293039A029B42EA030343F08D
:1031C00004030293029BDBB203F03F03019A82F8EF
:1031D000243005B000BD00BF00B585B00190134696
:1031E0000A468DF803208DF802304FF000038DF869
:1031F0000F30019A40F20003C4F201039A4207D053
:1032000044F66400C0F2000040F26E41FDF748FA57
:103210009DF80330002B0BD09DF80330012B07D015
:1032200044F66400C0F2000040F26F41FDF738FA46
:103230009DF80230002B0BD09DF80230012B07D0F7
:1032400044F66400C0F200004FF48E61FDF728FAE6
:103250009DF80330002B02D0012B05D008E04FF081
:1032600001038DF80F3003E04FF002038DF80F30AB
:103270009DF80230012B0AD1019B1B7CDAB29DF82C
:103280000F3042EA0303DAB2019B1A7411E0019B8A
:103290001B7CDBB21A469DF80F306FEA0303DBB2EA
:1032A000DBB203F0F30302EA0303DBB2DAB2019B01
:1032B0001A7405B000BD00BF00B585B0019013467B
:1032C0000A468DF803208DF80230019A40F200037F
:1032D000C4F201039A4207D044F66400C0F2000031
:1032E00040F29641FDF7DCF99DF80330002B0FD03A
:1032F0009DF80330012B0BD09DF80330022B07D033
:1033000044F66400C0F2000040F29741FDF7C8F9AE
:103310009DF80230002B0BD09DF80230012B07D016
:1033200044F66400C0F200004FF49361FDF7B8F971
:103330009DF80330012B08D0022B0BD0002B0DD1B0
:103340004FF010038DF80F3008E04FF040038DF878
:103350000F3003E06FF07F038DF80F309DF80230DF
:10336000012B0AD1019B1B7CDAB29DF80F3042EA97
:103370000303DAB2019B1A7411E0019B1B7CDBB2E0
:103380001A469DF80F306FEA0303DBB2DBB203F09D
:10339000F30302EA0303DBB2DAB2019B1A7405B04D
:1033A00000BD00BF00B583B00190019A40F2000358
:1033B000C4F201039A4207D044F66400C0F2000050
:1033C00040F2C141FDF76CF9019B1B7EDBB2184650
:1033D00003B000BD00B585B001900091019A40F2A4
:1033E0000003C4F201039A4207D044F66400C0F21D
:1033F000000040F2D541FDF753F9009B9B78002B6C
:103400000BD0009B9B78012B07D044F66400C0F2E0
:10341000000040F2D641FDF743F9009BDB78002B1A
:103420000BD0009BDB78012B07D044F66400C0F280
:10343000000040F2D741FDF733F9009BDB79FF2B09
:1034400007D144F66400C0F200004FF49B61FDF721
:1034500027F9009B5B79002B0BD0009B5B79012B3C
:1034600007D044F66400C0F2000040F2D941FDF7F5
:1034700017F9009B1B79002B0BD0009B1B79012BAC
:1034800007D044F66400C0F2000040F2DA41FDF7D4
:1034900007F9009B9B79FF2B07D144F66400C0F22B
:1034A000000040F2DB41FDF7FBF8009B1B78002B8E
:1034B0000BD0009B1B78012B07D044F66400C0F2B0
:1034C000000040F2DC41FDF7EBF8009B5B78002B3D
:1034D0000BD0009B5B78012B07D044F66400C0F250
:1034E000000040F2DD41FDF7DBF84FF000030393ED
:1034F000009BDB78012B18D1039B43F0100303934F
:10350000009B5B79012B03D1039B43F020030393C2
:10351000009B1B79012B03D1039B43F0080303930A
:10352000009BDA79019B83F85420009B1B78012BC8
:1035300003D1039B43F001030393009B9B78012B72
:1035400008D1039B43F004030393009B9A79019BEA
:1035500083F85020009B5B78002B03D1039B43F042
:1035600002030393039BDBB203F03F03019A82F84B
:103570004C30019B1B7BDBB243F03803DAB2019B7A
:103580001A7305B000BD00BF82B001900B468DF8E4
:1035900003309DF80330012B09D1019B93F84C3087
:1035A000DBB203F0FD03019A82F84C3009E0019B85
:1035B00093F84C30DBB243F00203DAB2019B83F89C
:1035C0004C2002B0704700BF00B587B00390029155
:1035D00001928DF803309DF80330002B27D0039B18
:1035E0001B7B8DF812309DF812308DF813309DF84A
:1035F000123023F010038DF81230039B9DF8122037
:103600001A73039B18460299019A4FF00103FFF7C2
:1036100003F803460593039B1B7DDBB203F04003D5
:10362000002BF8D0039B9DF813201A7310E0039B26
:1036300018460299019A4FF00103FEF7EDFF034689
:103640000593039B1B7DDBB203F04003002BF8D0F6
:10365000059B184607B000BD00B583B001900B462E
:103660008DF803300DF10303019819464FF0010264
:103670004FF00103FFF7A8FF03B000BD00B585B010
:1036800003900291019203980299019A4FF000036E
:10369000FFF79AFF0346184605B000BD4CF2000341
:1036A000C4F20F03D3F888304FEA136303F0030327
:1036B000032B40F0AA804CF20003C4F20F03D3F8AE
:1036C0000C3103F00303032B00F2F48001A252F843
:1036D00023F000BFE536000049370000AF37000097
:1036E000E53600004CF20003C4F20F03D3F8883033
:1036F0004FEA43434FEA534303F1010241F20023EF
:10370000C0F27A0303FB02F24CF20003C4F20F038F
:10371000D3F888304FEA134303F0FF0303F10103AA
:10372000B2FBF3F24CF20003C4F20F03D3F80431FE
:1037300003F0FF0303F10103B2FBF3F240F2AC1319
:10374000C1F200031A60B6E04CF20003C4F20F03AA
:10375000D3F888304FEA43434FEA534303F1010261
:1037600043F20063C0F26E1303FB02F24CF200035B
:10377000C4F20F03D3F888304FEA134303F0FF037A
:1037800003F10103B2FBF3F24CF20003C4F20F03A6
:10379000D3F8043103F0FF0303F10103B2FBF3F2AA
:1037A00040F2AC13C1F200031A6000BF83E04CF298
:1037B0000003C4F20F03D3F888304FEA43434FEAC3
:1037C000534303F101034FEA03424CF20003C4F2F6
:1037D0000F03D3F888304FEA134303F0FF0303F1DC
:1037E0000103B2FBF3F24CF20003C4F20F03D3F86F
:1037F000043103F0FF0303F10103B2FBF3F240F2E3
:10380000AC13C1F200031A6055E04CF20003C4F29D
:103810000F03D3F80C3103F00303032B4BD801A2A1
:1038200052F823F035380000613800008D38000070
:10383000353800004CF20003C4F20F03D3F8043112
:1038400003F0FF0303F1010240F60013C0F23D0351
:10385000B3FBF2F240F2AC13C1F200031A602AE0AB
:103860004CF20003C4F20F03D3F8043103F0FF035A
:1038700003F1010241F60033C0F2B703B3FBF2F2E9
:1038800040F2AC13C1F200031A6014E04CF20003E2
:10389000C4F20F03D3F8043103F0FF0303F1010373
:1038A0004FF40042B2FBF3F240F2AC13C1F200035A
:1038B0001A6000E000BF70474CF20003C4F20F032F
:1038C0004FF02002C3F8A0214CF20003C4F20F0312
:1038D000D3F8A03103F02003002B09D04CF20003F1
:1038E000C4F20F03D3F8A03103F04003002BF5D04E
:1038F0004CF20003C4F20F034FF00302C3F804219B
:103900004CF20003C4F20F034FF00002C3F8A821E9
:103910004CF20003C4F20F034FF00002C3F8AC21D5
:103920004CF20003C4F20F034FF00102C3F80C2164
:103930004CF20003C4F20F0340F26302C0F205022E
:10394000C3F884204CF20003C4F20F034FF0AA0224
:10395000C3F88C204CF20003C4F20F034FF0550261
:10396000C3F88C204CF20003C4F20F034FF00102A5
:10397000C3F880204CF20003C4F20F034FF0AA02F8
:10398000C3F88C204CF20003C4F20F034FF0550231
:10399000C3F88C204CF20003C4F20F03D3F8883034
:1039A00003F08063002BF5D04CF20003C4F20F0348
:1039B0004FF00302C3F880204CF20003C4F20F035F
:1039C0004FF0AA02C3F88C204CF20003C4F20F039C
:1039D0004FF05502C3F88C204CF20003C4F20F03E1
:1039E000D3F8883003F04073002BF5D04CF200037D
:1039F000C4F20F034FF02302C3F8A4204CF20003DB
:103A0000C4F20F034FF0AA02C3F8AC204CF200033B
:103A1000C4F20F034FF05502C3F8AC204CF2000380
:103A2000C4F20F034FF00102C3F8A0204CF20003D0
:103A3000C4F20F034FF0AA02C3F8AC204CF200030B
:103A4000C4F20F034FF05502C3F8AC204CF2000350
:103A5000C4F20F03D3F8A83003F48063002BF5D031
:103A60004CF20003C4F20F034FF00302C3F8A0208E
:103A70004CF20003C4F20F034FF0AA02C3F8AC20CB
:103A80004CF20003C4F20F034FF05502C3F8AC2010
:103A90004CF20003C4F20F03D3F8A83003F44073D0
:103AA000002BF5D04CF20003C4F20F0348F2DE7293
:103AB000C0F22842C3F8C4204CF20003C4F20F0342
:103AC0004FF00002C3F8C8214CF20003C4F20F0308
:103AD00043F23A021A604EF60053CEF200034FF062
:103AE00000029A60704700BF84B001900091019B72
:103AF0001F2B03D9019BA3F1200300E0019B03933B
:103B0000019B1F2B27D84CF20003C4F20F034CF289
:103B10000002C4F20F02D2F8A811039A4FF003007A
:103B200000FA02F26FEA020201EA0202C3F8A821D7
:103B30004CF20003C4F20F034CF20002C4F20F0275
:103B4000D2F8A811039A009800FA02F241EA0202A0
:103B5000C3F8A82126E04CF20003C4F20F034CF294
:103B60000002C4F20F02D2F8AC11039A4FF0030026
:103B700000FA02F26FEA020201EA0202C3F8AC2183
:103B80004CF20003C4F20F034CF20002C4F20F0225
:103B9000D2F8AC11039A009800FA02F241EA02024C
:103BA000C3F8AC2104B0704784B00190019B1F2B77
:103BB00009D8019B02934CF20003C4F20F03D3F81F
:103BC000A83103930AE0019BA3F1200302934CF276
:103BD0000003C4F20F03D3F8AC310393029B039AA2
:103BE00022FA03F303F003030393039B184604B084
:103BF000704700BF00B585B0019040F2AC13C1F230
:103C000000031B6802930198FFF7CEFF034603935E
:103C1000039B032B19D801A252F823F02D3C00007E
:103C2000353C00003D3C0000453C00004FF00403E3
:103C300003930AE04FF00103039306E04FF0020301
:103C4000039302E04FF008030393029A039BB2FB35
:103C5000F3F30293029B184605B000BD82B00190B9
:103C60000B468DF803309DF80330012B15D14CF233
:103C70000002C4F20F024CF20003C4F20F03D3F8A7
:103C8000C41001984FF2DE73CEF6EF7300EA03031F
:103C900041EA0303C2F8C4301AE09DF80330002B58
:103CA00016D14CF20002C4F20F024CF20003C4F22F
:103CB0000F03D3F8C410019B6FEA030301EA030169
:103CC0004FF2DE73CEF6EF7301EA0303C2F8C4309D
:103CD00002B070474CF20003C4F20F034FF0000231
:103CE000C3F8C02030BF70474EF60053CEF2000339
:103CF0004FF004021A614CF20003C4F20F034FF0BC
:103D00000802C3F8C02030BF704700BF4EF6005312
:103D1000CEF200034FF004021A614CF20003C4F229
:103D20000F034FF00902C3F8C02030BF704700BF37
:103D30004EF60053CEF200034FF004021A614CF22B
:103D40000003C4F20F034FF00302C3F8C02030BFDA
:103D5000704700BF4BB942B9002908BF002802D004
:103D60004FF0FF31084600F037B882B0EC462DE93D
:103D7000005000F005F8DDF804E002B00CBC70471C
:103D8000F8B514461D4606460F4600F0D9F900FB6B
:103D900005F5A0FB042304FB0154E318B61A67EBF6
:103DA0000307069BC3E90067F8BD00BFF8B51446DA
:103DB0001D4606460F4600F011F800FB05F5A0FB76
:103DC000042304FB0154E318B61A67EB0307069BB0
:103DD000C3E90067F8BD00BF704700BF00292DE9A7
:103DE000F04F85B0C0F2C8800026002BC0F2BF8023
:103DF0008946144605469B46002B4AD18A4257D92C
:103E0000B2FA82F353B1C3F1200001FA03F925FAA3
:103E100000F812FA03F49D4048EA0909270C4846C5
:103E200039461FFA84FB00F00BFB394682464846B0
:103E300000F034FC2A0C0BFB0AF342EA01494B4523
:103E400009D919EB04090AF1FF3A04D24B4584BFA2
:103E50000AF1FF3AA144C3EB090939464846ADB21D
:103E600000F0EEFA39468046484600F017FC0BFB9E
:103E700008FB45EA0145AB4507D92D1908F1FF3884
:103E800003D2AB4588BF08F1FF3848EA0A4800274B
:103E900003E08B4257D90027B84642463B4616B14D
:103EA000524263EB43031946104605B0BDE8F08F5C
:103EB00022B91146012000F0C3FA0446B4FA84F88E
:103EC000B8F1000F5ED1C4EB0908270C1FFA84F982
:103ED000012102913946404600F0B2FA3946824645
:103EE000404600F0DBFB4FEA154809FB0AF348EABD
:103EF000014B5B4509D91BEB040B0AF1FF3A04D2D5
:103F00005B4584BF0AF1FF3AA344C3EB0B0B394670
:103F10005846ADB200F094FA39468046584600F053
:103F2000BDFB09FB08F945EA0145A94507D92D194B
:103F300008F1FF3803D2A94588BF08F1FF3848EAE5
:103F40000A48029FA9E7B3FA83F7002F68D18B4292
:103F50002CBF4FF000094FF0010982428CBF4C4644
:103F600049F00104002C96D04FF0010895E7524229
:103F700063EB4303F6433BE7404261EB41014FF003
:103F8000FF3632E704FA08F4C8F1200735FA07F3E0
:103F900029FA07FA270C09FA08FB3946504643EA82
:103FA0000B02029200F04CFA39461FFA84F983465C
:103FB000504600F073FB029809FB0BF2030C43EA36
:103FC00001439A4204D91B190BF1FF3BC0F0B180A9
:103FD0009B1A39461846019300F032FA019982463D
:103FE0000846394600F05AFBDDF808C009FB0AF321
:103FF0001FFA8CF040EA0142934208D912190AF1E3
:10400000FF3A04D2934284BF0AF1FF3A121905FA2B
:1040100008F54AEA0B4EC3EB0208CDF808E059E771
:10402000C7F1200003FA07FAC24035FA00F342EA6A
:104030000A0B21FA00F801FA07F940464FEA1B4A39
:1040400043EA0901029151461FFA8BF2039200F0F4
:10405000F7F951468146404600F020FB039BDDF80E
:1040600008C003FB09F24FEA1C4014FA07F340EAC8
:104070000144A24204D914EB0B0409F1FF3952D3D5
:10408000A41A51462046019300F0DAF951468046C1
:10409000204600F003FB0398DDF808C000FB08F29F
:1040A0001FFA8CF343EA0140019B824204D910EBD2
:1040B0000B0008F1FF3830D348EA09481FFA83FCA7
:1040C0001B0C801A1FFA88FE4FEA184A0CFB0EF9E7
:1040D0000CFB0AFC03FB0EC103FB0AF201EB1941C6
:1040E0008C4588BF02F5803202EB114E704510D32B
:1040F0001FFA89F905FA07F709EB014014BF0022FE
:10410000012287422CBF002702F00107002F3FF455
:10411000C4AE08F1FF380027BFE6824284BF58448E
:1041200008F1FF38C8E7A24284BF09F1FF395C44B7
:10413000A6E79A4284BF0BF1FF3B1B1948E700BF7B
:104140002DE9F04F0C4683B08046164689461F463F
:1041500015468A46002B4BD18A425CD9B2FA82F3CB
:104160005BB1C3F1200001FA03FA28FA00F216FA53
:1041700003F508FA03F842EA0A0A2E0C50463146C3
:10418000AFB200F05DF931464FEA1844814650461F
:1041900000F084FA07FB09F344EA014A534509D9C0
:1041A0001AEB050A09F1FF3904D2534584BF09F11E
:1041B000FF39AA44C3EB0A0A314650461FFA88F871
:1041C00000F03EF931460446504600F067FA07FB1E
:1041D00004F748EA0148474506D9013C18EB0508B1
:1041E00002D2474588BF013C44EA094400265CE00E
:1041F0008B4258D8B3FA83F6002E5BD18B422CBF8A
:104200000022012285428CBF154642F00105002D97
:1042100049D0012449E022B91146012000F010F9EB
:104220000546B5FA85F6002E40F0BA80641B2F0CC7
:104230001FFA85FA01263946204600F001F9394671
:104240004FEA184B8146204600F028FA0AFB09F392
:104250004BEA014B5B4509D91BEB050B09F1FF3913
:1042600004D25B4584BF09F1FF39AB44C3EB0B0BB0
:10427000394658461FFA88F800F0E2F839460446F5
:10428000584600F00BFA0AFB04FA48EA0148C24516
:1042900006D9013C18EB050802D2C24588BF013C93
:1042A00044EA094401E0002634463146204603B082
:1042B000BDE8F08FC6F12000B34032FA00F721FAD2
:1042C00000FB1F4314FA06F228FA00F158464FEAA1
:1042D000174A114300915146BBB2019300F0B0F868
:1042E0005146B5408146584600F0D8F9019C0098E7
:1042F00004FB09F34FEA104C4CEA014B5B4505D92E
:104300001BEB070B09F1FF39C0F08E80C3EB0B0BE1
:104310005146584600F094F851460446584600F07D
:10432000BDF90198009A00FB04F31FFA82FC4CEAE5
:104330000142934206D9013CD21903D2934201D9DA
:10434000D219013C44EA0944A8B2D21A2D0C1FFA32
:1043500084FC230C00FB0CF700FB03FE05FB0CE1C7
:1043600005FB03F501EB17418E4588BF05F5803548
:1043700005EB1145AA4210D3BFB208FA06F607EBC7
:10438000014214BF4FF0000E4FF0010E96422CBFB9
:1043900000260EF00106002E87D0013C002684E79F
:1043A000B540C6F1200124FA01F928FA01F22F0CD8
:1043B000B440394648462243009200F041F839465D
:1043C0001FFA85FA8346484600F068F9009B1A0CEC
:1043D0000AFB0BF342EA0144A34203D964190BF12F
:1043E000FF3B27D3E41A3946204600F029F8394626
:1043F0008146204600F052F900980AFB09F31FFAA3
:1044000080FC4CEA0144A34208D9641909F1FF3940
:1044100004D2A34284BF09F1FF39641908FA06F8EF
:10442000E41A49EA0B4606E75B4584BF09F1FF3908
:10443000BB446BE7A34284BF0BF1FF3B6419D1E798
:104440004A1E08BF7047C0F02481884240F216819E
:10445000114200F01781B0FA80F3B1FA81F2A2EBB9
:104460000303C3F11F0304A202EB03134FF0000286
:104470009F4600BFAFF30080B0EBC17F00BF42EBAF
:10448000020228BFA0EBC170B0EB817F00BF42EBFE
:10449000020228BFA0EB8170B0EB417F00BF42EB6E
:1044A000020228BFA0EB4170B0EB017F00BF42EBDE
:1044B000020228BFA0EB0170B0EBC16F00BF42EB5E
:1044C000020228BFA0EBC160B0EB816F00BF42EBDE
:1044D000020228BFA0EB8160B0EB416F00BF42EB4E
:1044E000020228BFA0EB4160B0EB016F00BF42EBBE
:1044F000020228BFA0EB0160B0EBC15F00BF42EB3E
:10450000020228BFA0EBC150B0EB815F00BF42EBBD
:10451000020228BFA0EB8150B0EB415F00BF42EB2D
:10452000020228BFA0EB4150B0EB015F00BF42EB9D
:10453000020228BFA0EB0150B0EBC14F00BF42EB1D
:10454000020228BFA0EBC140B0EB814F00BF42EB9D
:10455000020228BFA0EB8140B0EB414F00BF42EB0D
:10456000020228BFA0EB4140B0EB014F00BF42EB7D
:10457000020228BFA0EB0140B0EBC13F00BF42EBFD
:10458000020228BFA0EBC130B0EB813F00BF42EB7D
:10459000020228BFA0EB8130B0EB413F00BF42EBED
:1045A000020228BFA0EB4130B0EB013F00BF42EB5D
:1045B000020228BFA0EB0130B0EBC12F00BF42EBDD
:1045C000020228BFA0EBC120B0EB812F00BF42EB5D
:1045D000020228BFA0EB8120B0EB412F00BF42EBCD
:1045E000020228BFA0EB4120B0EB012F00BF42EB3D
:1045F000020228BFA0EB0120B0EBC11F00BF42EBBD
:10460000020228BFA0EBC110B0EB811F00BF42EB3C
:10461000020228BFA0EB8110B0EB411F00BF42EBAC
:10462000020228BFA0EB4110B0EB011F00BF42EB1C
:10463000020228BFA0EB0110B0EBC10F00BF42EB9C
:10464000020228BFA0EBC100B0EB810F00BF42EB1C
:10465000020228BFA0EB8100B0EB410F00BF42EB8C
:10466000020228BFA0EB4100B0EB010F00BF42EBFC
:10467000020228BFA0EB0100104670470CBF0120CA
:1046800000207047B1FA81F2C2F11F0220FA02F055
:10469000704708B14FF0FF30FFF79EBB0029F8D0FC
:1046A0002DE90340FFF7CCFEBDE8064002FB00F316
:1046B000A1EB0301704700BF08B500F04BF80748B5
:1046C00000B10068064901B109680022FBF7E2FF6A
:1046D000044B0BB1AFF30080FEE700BF0000000009
:1046E000000000000000000080B51448144B21E0D9
:1046F0005C689968DD688C420CD0002205E0A61841
:104700000832D6E9008941E902898C460831AA427B
:10471000F5D101E004EB050C1C696146002204E0C0
:1047200008320026002741E902670831A242F7D18A
:10473000143301380028DBD1FFF7BEFF0100000071
:104740009448000001498D46014908470080001047
:10475000E946000070B544F6800644F68005C0F2D4
:104760000006C0F20005761BB61006D0002455F8EE
:10477000243001349847A642F9D844F6800544F61F
:104780008406C0F20005C0F20006761B00F072F845
:10479000B61006D0002455F8243001349847A642BC
:1047A000F9D870BD0A0D506C6561736520696E7033
:1047B0007574206672657175656E637920286672FE
:1047C0006F6D203120746F2039393920687A293A89
:1047D000000000002E2E2E506C6561736520696EFE
:1047E000707574206469676974732066726F6D20D8
:1047F0003020746F2039206F6E6C7921000000002A
:104800000A0D4D6561737572696E672E2E2E2E2E00
:104810002E000000687A00000A0D50726573732044
:104820006320746F20636F6E74696E7565206D65AB
:1048300061737572696E67206F7468657220736941
:10484000676E616C732E2E2E000000000A0D0000B2
:10485000307800006C7063313778785F74696D650B
:10486000722E63006C7063313778785F7561727493
:104870002E630000F8B500BFF8BC08BC9E46704728
:10488000F1000000F8B500BFF8BC08BC9E467047B8
:10489000DD00000000000000B04800000000001033
:0848A000B0010000400000001F
:0848A80024B8FF7F01000000AD
:1048B00000000000000000002A2A2A2A2A2A2A2AA8
:1048C0002A2A2A2A2A2A2A2A2A2A2A2A2A2A2A2A48
:1048D0002A2A2A2A2A2A2A2A2A2A2A2A2A2A2A2A38
:1048E0002A2A2A2A2A2A2A2A2A2A2A2A2A2A2A2A28
:1048F0002A2A2A2A2A2A2A2A2A2A2A2A2A2A2A2A18
:104900002A2A2A2A2A2A2A2A0A0D4C696E636F6CDF
:104910006E203630200A0D54696D6572206D656118
:1049200073757265206672657175656E6379206452
:10493000656D6F200A0D09202D204D43553A204CFE
:10494000504331377878200A0D09202D20436F72AB
:10495000653A2041524D20436F727465782D4D3376
:10496000200A0D09202D20436F6D6D756E696361FE
:104970007465207669613A20434F4D31202D202007
:1049800031313532303020627073200A0D2055737A
:10499000652074696D6572203020746F206D6561CB
:1049A0007375726520696E707574207369676E61C6
:1049B0006C206672657175656E6379207468726FBC
:1049C0007567682069747320434150302E30200A87
:1049D0000D205573652074696D6572203220746FE7
:1049E0002067656E657261746520646966666572CC
:1049F000656E74206672657175656E637920736982
:104A0000676E616C73200A0D2A2A2A2A2A2A2A2A0A
:104A10002A2A2A2A2A2A2A2A2A2A2A2A2A2A2A2AF6
:104A20002A2A2A2A2A2A2A2A2A2A2A2A2A2A2A2AE6
:104A30002A2A2A2A2A2A2A2A2A2A2A2A2A2A2A2AD6
:104A40002A2A2A2A2A2A2A2A2A2A2A2A2A2A2A2AC6
:104A50002A2A2A2A2A2A2A2A0A0D000000E1F50514
:00000001FF
